:0200000480007A
:100000006F008004732F2034930F80006308FF0378
:10001000930F90006304FF03930FB0006300FF038E
:10002000130F000063040F0067000F00732F2034CC
:1000300063540F006F00400093E19153171F0000BD
:1000400023223FFC6FF09FFF93000000130100008C
:10005000930100001302000093020000130300004C
:100060009303000013040000930400001305000034
:10007000930500001306000093060000130700001C
:100080009307000013080000930800001309000004
:1000900093090000130A0000930A0000130B0000EC
:1000A000930B0000130C0000930C0000130D0000D4
:1000B000930D0000130E0000930E0000130F0000BC
:1000C000930F0000732540F16310050097020000B4
:1000D000938202017390523073500018970200000F
:1000E00093824202739052309B021000939252030B
:1000F0009382F2FF7390023B9302F0017390023AF5
:100100007350403097020000938242017390523046
:10011000735020307350303093010000970200007C
:10012000938282EE73905230130510001315F5017F
:10013000635C05000F00F00F930110009308D005D9
:10014000130500007300000093020000638A0200A0
:1001500073905210B7B200009B82921073902230BD
:100160007350003097020000938242017390123462
:10017000732540F1730020309300000013B7000096
:100180009303000093012000631277269300100070
:1001900013B7100093030000930130006318772415
:1001A0009300300013B770009303100093014000D8
:1001B000631E77229300700013B730009303000092
:1001C00093015000631477229300000013B700805E
:1001D0009303100093016000631A7720B70000803A
:1001E00013B70000930300009301700063107720A1
:1001F000B700008013B700809303100093018000C4
:100200006316771E9300000013B7F07F930310006E
:1002100093019000631C771CB70000809B80F0FF67
:1002200013B70000930300009301A0006310771C34
:10023000B70000809B80F0FF13B7F07F93030000AE
:100240009301B0006314771AB700008013B7F07FF2
:10025000930300009301C000631A7718B700008071
:100260009B80F0FF13B70080930310009301D00030
:10027000631E77169300000013B7F0FF930310007E
:100280009301E000631477169300F0FF13B710009A
:10029000930300009301F000631A77149300F0FFBA
:1002A00013B7F0FF9303000093010001631077146C
:1002B0009300B00093B0D00093031000930110019D
:1002C00063967012130200009300F00013B7A000B1
:1002D000130307001302120093022000E31652FEDC
:1002E00093030000930120016312731013020000B6
:1002F0009300A00013B700011300000013030700D0
:100300001302120093022000E31452FE9303100024
:1003100093013001631C730C130200009300000171
:1003200013B7900013000000130000001303070030
:100330001302120093022000E31252FE9303000006
:10034000930140016314730A130200009300B0008C
:1003500013B7F0001302120093022000E31852FEBC
:1003600093031000930150016312770813020000F9
:10037000930010011300000013B780001302120055
:1003800093022000E31652FE9303000093016001E4
:10039000631E7704130200009300C00013000000E6
:1003A0001300000013B7E0001302120093022000B4
:1003B000E31452FE93031000930170016318770257
:1003C0009330F0FF9303100093018001639070025B
:1003D000B700FF009B80F00F13B0F0FF9303000005
:1003E0009301900163147000631030020F00F00F4E
:1003F000638001009391110093E111009308D005EF
:1004000013850100730000000F00F00F930110002E
:100410009308D0051305000073000000731000C09E
:1004200000000000000000000000000000000000CC
:0C043000000000000000000000000000C0
:1010000000000000000000000000000000000000E0
:1010100000000000000000000000000000000000D0
:1010200000000000000000000000000000000000C0
:1010300000000000000000000000000000000000B0
:081040000000000000000000A8
:040000058000000077
:00000001FF
